:1000000011298030A100FE30AF200130AF207530C3
:10001000A7003030C628A101A117AF00AF08031D0B
:100020001328030114280130AF020310A20CA20C04
:10003000A20CC0302205403EAF07FE30AF202F0893
:10004000AF28A101A117AF00FE30AF202F08AF28C5
:10005000A401AA00AB01A01124080319A0150530C2
:10006000A3002730A900103041200330A900E83058
:100070004120A90164304120A9010A3041202A0809
:100080004828A8002B08A7002A08A600DA2026087E
:10009000A600A3030319A011240803195228230260
:1000A000031859282608031DA011A0195928303E0D
:1000B000AF280800A300240803190C292308AF2047
:1000C000A4035B28AD000611861183160611861164
:1000D0000F30860583122D08A0188C283E30A7000B
:1000E0008030C6203330AC00A0201330A700883009
:1000F000C620A0206430C520A0206430C520223056
:10010000AC00A02028308B200C308B2006308B20B8
:10011000A0142D088C282014AC00201C9A288611CD
:10012000033C031C9F289F200530A700DC30C6201D
:10013000031408002014FE3C0319AD288615201C6A
:10014000201006150F3086052C08F039860406119C
:10015000AC0E2018A0283230C5202D080C29A11B78
:10016000622883178001840AFF3E031DB2280C29F0
:10017000A901A800FF30A807031CA907031C0C292C
:100180000330A700DF30C620BA28A701E83EA6004A
:10019000A709FC30031CCF28A6070318CC28A60704
:1001A0000000A70FCC282618D528A61CD9280000A7
:1001B000D9280800AB01AA011030AC00270DAA0D08
:1001C000AB0D2808AA022908031C290FAB0203184B
:1001D000F0282808AA0729080318290FAB070310DD
:1001E000A60DA70DAC0BDE2826080C291030B00098
:1001F000A701A601AD0CAC0C031C04292808A60716
:1002000029080318290FA707A70CA60CAB0CAA0CEA
:10021000B00BFA282A080C29831383120313000059
:100220000800A00107309F00E03083168500FF30F2
:10023000860081138312850186012030840060309E
:10024000B220A03084005030B22020308400303002
:10025000B120C830B82001207730622062206220AF
:100260002E3062207030622069306220633062205C
:100270006230622061306220733062206930622017
:10028000633062202E3062206E3062206C3062203B
:100290000B30A900B830B92001204430622043302F
:1002A00062204630622031306220363062204E308B
:1002B00062204C3062204430622020306220622074
:1002C000563062202D306220323062200730A90083
:1002D000D030B92001204C306220443062205230AE
:1002E00062202030622061306220663062207230ED
:1002F00062206530622067306220653062206C3099
:100300006220653062206E30622086188D29851F3C
:100310008B2905148C290510852901205330622072
:1003200069306220673062206E3062206130622066
:1003300062206C306220203062207A3062206F3080
:100340006220653062206B306220653062206E3042
:10035000622036140512831605128312412AC30146
:100360003C03A500C90149082502031CC829EB214B
:10037000B61CC6294308A6004908A200A601A20A85
:100380000314A60DA20BC1292608C304C90FB32963
:10039000B2014308B100B20CB10CB20CB10CB20CFA
:1003A000B10CB20CB10C0F30B2053208AD003108FF
:1003B000AC00A9010A30A800F620B1002B08B20059
:1003C000B4014308B3000F30B3050030B405310861
:1003D0003307C3000800BA01B9010618002A01302A
:1003E000B820B90A0319BA0A0B303A02031CFF29D4
:1003F000031DFE29B9303902031CFF29372DED29D1
:100400009B30B8200618B614061CB610361C212ADC
:10041000440EB100B200F030B1050F30B205320821
:10042000A7003108A600A9013A30A800DA20BD00D3
:100430008030A1000230A2003D080D20FF30622074
:10044000342A8030A1000130A2003D080D20023086
:10045000A4004408292003013619013EB618013AC8
:1004600003193611031D3615C40A85140130A9007D
:10047000F430B9208510A901F030A8002808B9206F
:100480000800BB01C4013612361AE32ABA01B901C9
:10049000061C5B2AB90A0319BA0A0130B820AF302A
:1004A0003A02031C5A2A031D592AC9303902031C77
:1004B0005A2A372D482ABA01B9010618972AB90ACB
:1004C0000319BA0A0A30B82036188B2A39080B3AB1
:1004D0003A04031D762A8030A1000130A2003D08B5
:1004E0000D2035306220393062208A2A3908193AC5
:1004F0003A04031D7D2A85148A2A39084B3A3A04A6
:10050000031D842A85108A2A3908FA3A3A04031D01
:100510008A2A372D962A11303A02031C962A031D87
:10052000952A95303902031C962A372D5D2A4130D1
:100530003B02031C9C2A372DBB0A3A08031DA42A40
:1005400065303902031CA52A3616361CE22A3B0EFA
:10055000B100B200F030B1050F30B2053208A7008B
:100560003108A600A9014130A800DA20BD00803082
:10057000A100803021205330622069306220673032
:1005800062206E3062206130622062206C30622016
:100590002030622067306220653062207630622031
:1005A0006F3062206E3062206430622065306220DD
:1005B0006E3062208030A1000230A2003D080D2084
:1005C000FF306220442A361C0D2B01204930622066
:1005D0006E3062206930622074306220693062209F
:1005E000613062206C30622069306220733062209A
:1005F0006530622072306220653062206E30622089
:100600002E306220622062208030A100C030212084
:100610001030A4005F305A207C2B0730BD00013021
:10062000A2003D080B20A101B61D252B3B30410245
:1006300003181C2BC10A242BC101173045020318D3
:10064000232BC50A242BC501292B4208C1004608CB
:10065000C500051B392B4508031D312B0C30C70085
:10066000382B0D304502031C382B0C304502C700D7
:100670003E2B4508C7002030622062200A30470226
:100680000318442B203062208030A1004708282026
:100690003A3062200230A400410829203A3062201A
:1006A000303062206220051B652B0C304502031898
:1006B0005E2B613062206D306220622B70306220D0
:1006C0006D3062200D30BD00672B0F30BD0041083A
:1006D00003190130031D0301B5001E304102031947
:1006E0000130031D03013504B500013086180301F4
:1006F000350403197C2B0F2D361E0D2DEB210130F7
:10070000C9000F3049020318882BEB21C90F812B38
:100710003611B611EB21EB21EB21B61C912B051400
:10072000922B05101230C9001430490203189B2B7C
:10073000EB21C90F942BEB210730BC00AF214308FC
:10074000C200EB21361DA52BB6150630BC00AF212B
:100750004308C600EB21361DAE2BB6150630BC0093
:10076000AF214308BE000330BC00AF214308C800DE
:100770000530BC00AF214308C0000830BC00AF21E9
:100780004308BF00EB21361DC62BB615361CCC2BFB
:10079000B619CB2B36100120B6190C2D8030A100D4
:1007A000C03021201030A40020305A208030212079
:1007B000A10101304802031DE22B4D30622061305F
:1007C0006220172C02304802031DEB2B44306220BC
:1007D00069306220172C03304802031DF42B573078
:1007E00062206F306220172C04304802031DFD2B5D
:1007F000443062206F306220172C05304802031D00
:10080000062C5630622072306220172C06304802C7
:10081000031D0F2C5A30622061306220172C0730E4
:100820004802031D172C5A3062206F30622080303E
:10083000A100C03021203E08282020306220013055
:100840004002031D322C6A306220613062206E301B
:10085000622075306220613062207230622069301F
:100860006220F12C02304002031D472C66306220CA
:100870006530622062306220723062207530622002
:10088000613062207230622069306220F12C0330C6
:100890004002031D552C6D306220613062206220C1
:1008A0007230622074306220F12C04304002031D4B
:1008B000642C6130622070306220723062206930B6
:1008C00062206C306220F12C05304002031D6F2C39
:1008D0006D3062206530622069306220F12C063074
:1008E0004002031D7C2C6A306220753062206E301D
:1008F000622069306220F12C07304002031D892CF0
:100900006A306220753062206C306220693062206B
:10091000F12C08304002031D9E2C6130622075309E
:10092000622067306220753062207330622074303C
:1009300062207530622073306220F12C0930400251
:10094000031DB52C73306220653062207030622048
:1009500074306220653062206D3062206230622027
:100960006530622072306220F12C0A304002031D93
:10097000C82C6F3062206B306220743062206F3080
:100980006220623062206530622072306220F12C79
:100990000B304002031DDD2C6E3062206F30622070
:1009A00076306220653062206D30622062306220D5
:1009B0006530622072306220F12C0C304002031D41
:1009C000F12C643062206530622063306220653033
:1009D00062206D30622062306220653062207230A9
:1009E000622009304002031D002D20306220273094
:1009F00062208030A1000230A4003F0829200C2D85
:100A00002030622032306220303062208030A100FD
:100A10000230A4003F0829200E2D372D412A851FC2
:100A2000162D0512831605128312182D831605162E
:100A300083129B30B820410803190130031D0301C4
:100A4000B50001308618030135040319282D05155A
:100A5000851585140130A900F430B92005118511E0
:100A600085100130A9004A30B920C40A7F2B01202B
:100A7000473062206530622062206E306220203074
:100A800062207330622069306220673062206E30ED
:100A900062206130622062206C306220203084004D
:100AA0006030B220A03084005030B220203084006A
:100AB0003030B1200618B616061CB612030106180F
:100AC000013EB61A013C031D6B2DB70A0319B80A83
:100AD0000130B8205E2D0301B61A0130013A031926
:100AE000B612031DB61603010618013EB61A013CE4
:100AF000031D802DB70A0319B80A0130B820732DE1
:100B000003303802DE300319370203184E2D361435
:020B1000412A78
:02400E00503F21
:00000001FF
